:020000002CC012
:10000200A7C0FDCFFCCFFBCFFACF6CC07BC0F7CF30
:10001200F6CFF5CFF4CFF3CFF2CFF1CFF0CFEFCFD2
:10002200EECFEDCF1027E80364000A0001000010B4
:100032000001100001009001A00FE8030000000081
:1000420000000A00020060013800020062013A006A
:100052000A0004003C000000F894EE27ECBBF1E03B
:10006200FBBFEBBFE5BFF8E1F1BDE1BD8DE0A2E072
:10007200BB27ED938A95E9F780E094E0A0E6ED9343
:100082000197E9F7E6E4F0E085919591009761F038
:10009200A591B59105901590BF01F00105900D92C3
:1000A2000197E1F7FB01F0CFEFE5EDBFE4E0EEBF32
:1000B200C0E6D1E088C0E981F070EBBDE881EABD1D
:1000C200E8E1E9BFD5D0A881B981AE0FBF1FFD011C
:1000D200EF2FF0E0E9BDE0916001A881EA0FE8BDF1
:1000E20022960895EA93FA93EFB7EA939398F6016A
:1000F20031966F01E9B7EF7EE9BFE991EFBFF99160
:10010200E9911895BAD0D9D0C6D0939AE9E0F0E037
:10011200EC15FD0551F4D401A00FB11FA9D0AE1BFF
:10012200BF0BBA93AA93C7DF03C0E9B7E77FE9BF62
:10013200CCD03BC0E881E064E7B98BE18A95F1F766
:10014200369A349BFECF349AE4B1F5B121960895E4
:1001520094D0B1D0A0D0F801EA19FB099F0158014F
:10016200829902C0939801C0939A82991CC0E0912F
:100172006201F0916301E217F30710F4CC24DD244D
:10018200E8E0F0E0CE16DF0618F4F60131966F01D2
:10019200E8E0F0E0EC15FD0531F4F301E00FF11FAA
:1001A200FA93EA9388DF8CD02496E991EFBFF99114
:1001B200E991B991A9919991899179916991F9906E
:1001C200199009901895E0E0E7BBEFE3E8BBECE398
:1001D200E4BBE0E0E5BBE8EFE1BBE4E0E2BBE0E08A
:1001E200EFBDE2E0EEBDE0E0EDBDECBDE7BDE6BD9A
:1001F200EBBDEABDE9BDE8BDEBB7E064EBBFE1E012
:10020200E5BFE0E4EABFE7B9E7E8E6B97894959A92
:10021200E8EEF3E02F01E0E0EA938CDFE851FC4FD7
:100222003F01B09904C0E8EEF3E03DD0959AB19950
:1002320004C0E4E1F5E037D0969AB29904C0ECE844
:10024200F5E031D0979AB39904C0E3E1F6E02BD000
:10025200AA9AB49904C0E5E9F6E025D0AB9AB5991B
:1002620004C0EAE3F7E01FD0AC9A4201D4CFFFCF3B
:10027200E0916001F091610108950A921A92FA9256
:100282006A937A938A939A93AA93BA93EA93FA9384
:10029200EFB7EA930895ECB5AE2FEDB5FE2FE0E08F
:1002A200EA2B8F0108952F01E5B3E37EE5BBE2B3AC
:1002B200EF71E2BB08953A932A931A930A93089531
:1002C2003B812A8119810881089509911991089524
:00000001FF
